:1000000012C02DC02BC02AC029C028C027C026C0BE
:1000100025C024C023C022C021C020C01FC01EC0D4
:100020001DC01CC01BC011241FBECFE5D4E0DEBF25
:10003000CDBF11E0A0E6B0E0E2E5F3E002C005903C
:100040000D92AC3AB107D9F711E0ACEAB1E001C0CA
:100050001D92A33BB107E1F772D079C1D1CF1895BA
:10006000FC01009701F12091AC013091AD01832F8B
:100070008F708F3021F481E08093AE0102C0109226
:10008000AE018091AE01882329F083E08083218333
:10009000228309C082E08083932F80E0822B9283A9
:1000A0008183238334838091AC019091AD0190933F
:1000B000B0018093AF01089542E050E06FEA71E033
:1000C0008CEA91E037D10895C39A30E43A95F1F77C
:1000D000C39888E090E020E030E23A95F1F7C598C7
:1000E000220FB49B216030E23A95F1F7C59A01974F
:1000F00099F72093AC0188E090E030E23A95F1F76F
:10010000C598220FB49B216030E23A95F1F7C59A69
:10011000019799F72093AD0180E00895CF93CFB771
:10012000F894BB9ABD9ABC98C49AC59AC398CCDF80
:10013000CFBF80E0CF91089580EA91E00895CF93FA
:10014000DF93CDB7DEB76B970FB6F894DEBF0FBE67
:10015000CDBF89E287BB86E388BB14BA8FEF85BB2E
:100160008BEE81BB84E082BB829B07C081E08093E1
:10017000B2018091980185BB02C01092B20181E06A
:100180008093B2012FEF80E792E0215080409040B1
:10019000E1F700C0000086B38670BB24B3948630BC
:1001A00009F4B12CC9DF7C01DC011296ED91FC91C0
:1001B00013970995D7011696ED91FC911797CE01EB
:1001C00001960995B1100FC08FEF84BB85BB8A8162
:1001D0009B818034910529F08038910591F000E0F1
:1001E00013C002E011C014BA15BA8A819B8180380D
:1001F000910549F08115904811F003E005C005E034
:1002000003C001E001C004E081E08BBF82E08BBF4E
:1002100085B7816085BF85B78D7F85BF8BB78064CB
:100220008BBFB11001C0789488E0A82E99249394D4
:1002300010E0000F111F005A1F4F6E01ECE1CE0EAF
:10024000D11CB11027C01092B1018091B101882357
:10025000E1F38FE697E10197F1F700C00000FE019E
:100260007496A8E9B1E08A2D01900D928A95E1F784
:10027000829B06C09092B2018091980185BB02C01A
:100280001092B201E091B201F0E0E856FE4F808199
:1002900086BD0AC015BA8C89809584BBAFE5BAEEDD
:1002A0001197F1F700C00000D7011296ED91FC9173
:1002B00013970995D7011696ED91FC911797CE01EA
:1002C000019609954A815B81F801208131812B5F7C
:1002D0003F4FA0E060E070E012C084239523892B9B
:1002E00061F0F90133978081782BF9013297808191
:1002F000682BF90131978081A82B2B5F3F4FF901C3
:10030000359780819181009741F76C8B872F8C60A6
:100310008D8B6E8B8F8B688F7C63798FAA8F6370C8
:100320006B8FFE017496808180958193EC15FD059D
:10033000D1F787CFFB01DC0104C08D9101908019BA
:1003400021F441505040C8F7881B990B0895F89448
:02035000FFCFDD
:1003520057011601D500A8008A006C000400101095
:1003620010020008080801000404048000020202CE
:100372000080202020000000000004001010100265
:100382000008080801000404040080020202800040
:10039200202020000000000008002020200400107F
:1003A2001010020008080801000404040080020280
:1003B2000280000202020040020202400002020227
:1003C2000000000000008000010080000002000028
:1003D2004000001040000200000020000008001051
:1003E200000020100001000020000000040800208E
:1003F20020000400101000020000080001000004A8
:1004020000000000000000800002008000020000E6
:100412000040000008400000010000200000100021
:10042200100000201000010000200000000408005D
:10043200202000040010100002000008000100004B
:1004420004000000000000008002000080000002A2
:1004520000004000010040000000080020000010E1
:10046200001000002010000100002000000004081D
:10047200002020000400101000020000080001000B
:100482000004000000000000FFF3FFF3FFC3FFFFC2
:0C0492008E0064005C00300000000000E0
:101800000000000016B415BA0F93EF93FF930FB7C3
:101810000F9301E00093B1010091B20103950770AD
:101820000093B201E8E9F1E0E00F00E0F01F008171
:1018300006BD11240F910FBFFF91EF910F911895E5
:00000001FF
